:10000000C0C025C1CEC0CDC0CCC0CBC07EC7C9C08A
:10001000C8C0DCC0C6C04DC8C4C0C3C0C2C0C1C017
:10002000C0C0BFC0BEC0FE645A50463C322A262221
:100030001E1A171412100E0D0C0B0A0908070605DC
:10004000040302010020555342204D703320506CB0
:1000500061796572200A0063204B41444F20467746
:10006000566572312E30310020202053687574207F
:10007000446F776E20202020002020202057616BC5
:10008000652055702020202020004465746563742D
:1000900020566D75736963322E2E00202D2D3A2D5A
:1000A0002D002020203A202000200920204E6578B5
:1000B000742044697220202020002020202020204D
:1000C0004E65787420202020202000202020205001
:1000D000726576696F757320202020002020202013
:1000E0004E6F204469736B20202020200020205276
:1000F000656D6F7665204469736B20202000202099
:1001000020204469736B204F4B20202020200020AA
:1001100020496E73657274204469736B202020003F
:1001200020202020434D44204661696C202020205F
:100130000020566D32204E6F20526573706F6E73C3
:100140006500001F1F1F1F1F000010181C1E1C1819
:100150001000001B1B1B1B1B000002061A1A1A06AC
:100160000200030F0D090B1B180000001C1F1111CA
:100170001F001F11050D1F0C0400040E1F0A040AA6
:100180000A0011241FBECFE5D4E0DEBFCDBF11E0D1
:10019000A0E6B0E001C01D92A234B107E1F78CD90E
:1001A00038CB2ECF80933E01109240018FEF809389
:1001B0003A0184E083BF89B7816089BF85B78C7FAE
:1001C000816085BF8BB780648BBF08951F920F92AB
:1001D0000FB60F9211242F933F934F938F939F93BA
:1001E00020913C0130913D01809140018F5F8695C7
:1001F0008E3009F53033F8F080913A0187FF1BC04B
:10020000422F220F331F220F331F832F3F71209164
:100210003E01231711F027FF0EC0309339014F73B1
:100220004093380190E025E0969587952A95E1F76F
:10023000817080933A01109240019F918F914F916C
:100240003F912F910F900FBE0F901F9018951F9206
:100250000F920FB60F9211242F933F938F939F937A
:10026000909140019B31A8F582B712BE30913F01B9
:10027000992359F480B38695869580FD2AC0109203
:100280003D0110923C0130E08DE0292F2F5F883135
:1002900010F02F5F8D508950893020F085EE82BF9D
:1002A0002FEF12C020FF10C080913C0190913D01C2
:1002B000880F991F30FF816090933D0180933C012E
:1002C0002B3110F085EE82BF209340013F5F3093C9
:1002D0003F019F918F913F912F910F900FBE0F90F3
:1002E0001F901895282F662311F0C49A01C0C49856
:1002F000C59887B38F6087BB98B3907F822F829514
:100300008F70892B88BB979A00C097982F70292BE4
:1003100028BB979A00C097989F6098BB0895C4988F
:10032000C59A87B3807F87BB979A00C086B397989A
:1003300000C0979A00C096B3979883FDF0CF82E0F3
:1003400090E00197F1F7C498C59A87B3807F87BB87
:10035000979A00C096B3979800C0979A00C086B34A
:100360008F709295907F9798892B08951F93182FDF
:10037000D6DF812F60E0B6DF1F9108951F93182FFD
:10038000CEDF812F61E0AEDF1F910895662311F467
:10039000805801C08054EADF0895C1DF90E00895DD
:1003A00081E0E4DF089582E0E1DF08951F93182FD4
:1003B000B6DF1A3041F4803410F080E001C080E4F0
:1003C0008058D4DF03C0812F61E08CDF1F91089536
:1003D000CF93DF93EC0101C0E9DF89918823E1F736
:1003E000DF91CF910895CF93DF93EC0101C0DEDF61
:1003F000FE01219684918823D1F7DF91CF91089552
:100400001F93182F87B38F6087BBBC9ABD9A8F9AB2
:1004100080E89EE30197F1F7C19AC09A979A00C0CD
:10042000979880E893E10197F1F7979A00C0979821
:1004300080E490E0FC013197F1F7979A00C097981B
:10044000FC013197F1F7C098979A00C097980197EF
:10045000F1F788E28BDF88E089DFA2DF86E086DFC4
:10046000812F84DF1F9108955D9BFECF8CB9089585
:10047000982F8091E700877F8093E7005D9BFECFF8
:100480009CB95D9BFECF8DE08CB90895982F80912B
:10049000E700877F8093E7005D9BFECF9CB95D9B63
:1004A000FECF80E28CB95D9BFECF6CB95D9BFECF29
:1004B0008DE08CB90895982F5D9BFECF8EE18CB9AD
:1004C0005D9BFECF80E28CB95D9BFECF9CB95D9BAE
:1004D000FECF6CB95D9BFECF4CB95D9BFECF8DE02E
:1004E0008CB908959091E7009F7D9093E7008093E9
:1004F0002D018091E70080628093E700089590913C
:10050000E7009F779093E700809341018091E70097
:1005100080688093E700089580E061E037DF8AE833
:1005200090E061DF55E44DE020E23EE45D9BFECFCC
:100530005CB95D9BFECF4CB9C9010197F1F7809181
:100540006000823099F755E64DE020E23EE45D9B85
:10055000FECF5CB95D9BFECF4CB9C9010197F1F7A5
:1005600080916000833099F78091E700877F8093C6
:10057000E7005D9BFECF80E18CB95D9BFECF8DE0F7
:100580008CB980E593EC0197F1F78091E700877FC4
:100590008093E7005D9BFECF81E98CB95D9BFECF28
:1005A0008DE08CB980E593EC0197F1F75D9BFECF70
:1005B0008DE08CB988EE93E024E630E0F9013197C4
:1005C000F1F70197D9F780916000882351F461E039
:1005D000DDDE8EEF90E007DF8091E700846080939E
:1005E000E70080916000813059F480E061E0CEDE68
:1005F0008CED90E0F8DE8091E7008B7F8093E70040
:100600000895EF92FF92CF93DF937B01805CAEDE83
:10061000C0E0D0E0F701EC0FFD1FE4918E2FAEDEBD
:100620002196C830D105B1F7DF91CF91FF90EF90BF
:10063000089587FFC0C0883D09F4B1C0893D08F026
:1006400049C0803C09F4ABC0813CF8F48A3909F414
:100650007CC08B3950F48D3809F479C08E3809F498
:100660007AC08A3809F0AAC06EC08E3909F475C004
:100670008F3920F48D3909F0A1C06BC08C3B09F48F
:100680006EC08E3B09F09AC06CC08C3C09F477C0F8
:100690008D3C80F4853C09F462C0863C20F4813CAA
:1006A00009F08CC064C0883C09F465C0893C09F03D
:1006B00085C065C08F3C09F456C0803D20F48D3C58
:1006C00009F07CC060C0823D09F461C0833D09F03F
:1006D00075C061C08C3E09F454C08D3EE8F4813E83
:1006E00009F447C0823E50F48D3D09F460C0803E5D
:1006F00009F457C08A3D09F061C055C0853E89F1B3
:10070000863E20F4843E09F059C033C0883EA9F1EA
:10071000893E09F053C035C0853F50F4833FE8F56A
:100720008F3E19F1823FA9F18D3E09F047C02DC0DF
:100730008B3F30F4893FC8F5883F09F03FC031C096
:100740008D3FE1F536C083E5089583E7089584E59C
:10075000089584E708958AE508958AE708958CE46A
:1007600008958CE6089584E4089584E6089581E46C
:10077000089581E6089583E4089583E6089585E465
:10078000089585E6089589E4089589E608958EE43C
:1007900008958EE608958FE408958FE6089582E522
:1007A000089582E7089585E5089585E7089589E528
:1007B000089589E70895803208F480E208951F9330
:1007C0008091E70084FD15C080E061E0DFDD10E08E
:1007D00003C080811F5FEADDE12FF0E0EE59FF4F9B
:1007E00080818823B1F703C080E2E0DD1F5F103114
:1007F000D9F71F910895FF921F938091E70084FF1E
:1008000082C080E061E0C2DD809132018231A8F4D3
:100810001091320120EFF22EF10EE12FF0E0EE59AF
:10082000FF4F8081115005DFC1DD1F15B1F78091A9
:10083000E7008F7E8093E70066C08091E70085FD2A
:1008400062C08091E7008F7D8093E7008BE080930A
:100850002D018091E70080628093E7008091310153
:100860008F3080F01091310190EFF92EF10EE12FD1
:10087000F0E0EE59FF4F80811150DBDE97DD1F1550
:10088000B1F73CC0809131018823C9F4E091310176
:10089000F0E0EE59FF4F808189DD1091320181EF48
:1008A000F82EF10EE12FF0E0EE59FF4F808111504C
:1008B000C0DE7CDD1F15B1F78091320122C0F090BF
:1008C000310110E007C0F0E0EE59FF4F8081B1DE4A
:1008D0006DDD1F5FEF2DE11B80913101811798F7CE
:1008E000F090320109C0EF2DF0E0EE59FF4F80810A
:1008F000FA949FDE5BDD1F5F1031A9F78091310113
:100900008150809331011F91FF900895CF92DF9223
:10091000EF92FF921F937C018AE060E037DDC70110
:1009200060E777E162D7D82EC92EC70160E777E18B
:100930005CD7662311F480E202C0862F805D36DD2D
:100940008D2D9C2D68E572E050D7182FF92E8D2D36
:100950009C2D68E572E049D7862F805D27DD812FC9
:100960009F2D6CE370E041D7E82ED92E812F9F2D6B
:100970006CE370E03AD7862F805D18DD8AE316DDE0
:100980008E2D9D2D6AE070E030D7862F805D0EDDC4
:100990008E2D9D2D6AE070E028D7805D07DD1F91C8
:1009A000FF90EF90DF90CF9008951F93182F80E075
:1009B00060E0ECDC83E0FADC812F6AE00AD7282FC4
:1009C000812F07D7192F105D222321F0805DEEDCE7
:1009D000812F03C0812FEADC80E2E8DC80E2E6DCE4
:1009E0001F9108951F93182F84E060E0CFDC11233E
:1009F00021F484E0DBDC80E205C0113031F484E0D6
:100A0000D5DC86E0D3DC80E207C0123041F484E01C
:100A1000CDDC86E0CBDC87E0C9DC80E2C7DC1F915F
:100A200008958091E70081FF2BC08091E70087FD4A
:100A300027C08091E70086FF0CC08091E7008F7B84
:100A40008093E7008AE060E0A1DC82EA90E0CBDC02
:100A50000AC08091E70080648093E70080912B01B9
:100A600090912C0153DF8091E7008F778093E7000E
:100A700089E0809341018091E70080688093E700DE
:100A800008958091E9008E3179F096988091E9007F
:100A90008F5F8093E900E091E900F0E0EA5DFF4FAD
:100AA000E49188E86E2FF2DC8091E9007EDF089502
:100AB0008091E900882379F096988091E90081502F
:100AC0008093E900E091E900F0E0EA5DFF4FE491F6
:100AD00088E86E2FDBDC8091E90067DF0895809164
:100AE000E70080FF2BC0969880E061E04FDC8AEB46
:100AF00090E079DC8091E70081FF04C080E06CE049
:100B00004CE0D9DC8091E700877F8093E7005D9B14
:100B1000FECF85E28CB95D9BFECF8DE08CB98091D4
:100B2000E7008D7F8093E7008091E7008E7F8093C0
:100B3000E7008091E7008F7E8093E7000895809121
:100B4000E70080FF3EC0969880E061E01FDC8BEC00
:100B500090E049DC8091E70081FF04C080E06CE018
:100B60004CE0A9DC80912B0190912C01069768F450
:100B70008091E700877F8093E7005D9BFECF86E250
:100B80008CB95D9BFECF8DE08CB98091E700877FAB
:100B90008093E7005D9BFECF86E28CB95D9BFECF24
:100BA0008DE08CB98091E7008D7F8093E700809184
:100BB000E7008E7F8093E7008091E7008F7E80932F
:100BC000E700089596988091E70080FF2BC080E0B1
:100BD00061E0DCDB89EA90E006DC8091E70081FFE0
:100BE00004C080E06CE04CE066DC8091E700877F29
:100BF0008093E7005D9BFECF8EE88CB95D9BFECFB6
:100C00008DE08CB98091E7008D7F8093E700809123
:100C1000E7008E7F8093E7008091E7008F7E8093CE
:100C2000E7000895809135018F5F809335018091B1
:100C30003501833010F01092350180913501D2DEFC
:100C400008958091E70080FF28C096988091E70082
:100C500081FF04C080E06CE04CE02DDC8091E70077
:100C6000877F8093E7005D9BFECF80E28CB95D9B20
:100C7000FECF8DE08CB989E060E088DB80E096DB18
:100C80008BE990E0B0DB8091E7008E7F8093E700F6
:100C90008091E7008D7F8093E70008958091E700C1
:100CA00080FF3FC096988091E70081FF1DC0809132
:100CB000E700877F8093E7005D9BFECF8BE88CB9D0
:100CC0005D9BFECF8DE08CB989E060E05FDB81E069
:100CD0006DDB8091E7008D7F8093E70080912B0191
:100CE00090912C0113DE08958091E700877F809317
:100CF000E7005D9BFECF8BE88CB95D9BFECF8DE05E
:100D00008CB989E060E042DB82E050DB8091E70053
:100D100082608093E7008091E70080648093E70021
:100D200008958091E70082FF41C096988091350137
:100D3000882361F48091E700877F8093E7005D9BC3
:100D4000FECF81E28CB95D9BFECF1FC08091350143
:100D5000813061F48091E700877F8093E7005D9B9D
:100D6000FECF8AE88CB95D9BFECF0FC08091350124
:100D7000823069F48091E700877F8093E7005D9B74
:100D8000FECF8FE88CB95D9BFECF8DE08CB989E0FA
:100D900060E0FCDA81E00ADB8091E7008D7F8093E0
:100DA000E7008091E7008E7F8093E700089500FFC1
:100DB00027C047DF80E060E0E9DA85E490E013DBFC
:100DC00088E690E010DB80E197E224E630E0F9016C
:100DD0003197F1F70197D9F788E0C8DA88E893E10D
:100DE00024E630E0F9013197F1F70197D9F79698A9
:100DF000959A8091E7008F7E8093E7000E7F33C045
:100E00009598969A88E893E124E630E0F9013197C5
:100E1000F1F70197D9F78CE0A9DA80E060E0B6DA63
:100E200085E490E0E0DA89E790E0DDDA80E197E2BE
:100E300024E630E0F9013197F1F70197D9F76CDB3F
:100E4000E091E900F0E0EA5DFF4FE49188E86E2F61
:100E50001DDB8091E900A9DD80913501C3DD8EE0C5
:100E600080936000016088E0809330010B7F0895DB
:100E700080913A0187FD48C002FD0CC020913A01E3
:100E8000802F86958170332727FD309590E02817B5
:100E9000390739F180913801803271F0813228F4BC
:100EA0008C30A1F08E30A9F40FC0823259F082321A
:100EB00028F08B3371F404C082E009C083E007C0DE
:100EC00086E005C088E003C081E001C087E0809330
:100ED000360180913A018170880F902F9D7F092FF4
:100EE000082B80913801803119F0813131F402C032
:100EF00085E001C084E08093360188E08093300172
:100F00000B7F8FEF80933A0108951F920F920FB6D7
:100F10000F9211242F933F938F939F938091E8001A
:100F200081508093E8008091E800882309F04AC04E
:100F300083E08093E800A598AD9AAC98A49A00004D
:100F4000000000000000989902C091E00DC099993E
:100F500002C093E009C09A9902C092E005C09B9933
:100F600002C098E001C090E0A498AC9AAD98A59A10
:100F70000000000000000000989902C096E00EC03A
:100F8000999904C01092370194E008C09A9904C05E
:100F90001092370195E002C09B9B97E0A598AD9A0F
:100FA000992319F4109237010DC0809137019817D9
:100FB00019F41092360106C09093370180913701E1
:100FC0008093360102FD0BC080913001882331F0FF
:100FD0008091300181508093300101C00460809184
:100FE000E70087FF0FC080914101882331F0809195
:100FF000410181508093410105C08091E7008F77C6
:101000008093E7008091E70085FF0FC080912D015C
:10101000882331F080912D01815080932D0105C0EE
:101020008091E7008F7D8093E70000FF0DC09699C7
:101030000BC080916100882331F080916100815064
:101040008093610001C0969A00FF2AC02091E700BA
:101050002170802F869586958695817090E030E08E
:10106000822B932B892B41F080EE9EE290933401EA
:1010700080933301077F14C0809133019091340134
:1010800001979093340180933301809133019091C3
:101090003401892B29F487E080933601809337014E
:1010A0009F918F913F912F910F900FBE0F901F90A6
:1010B00018951F920F920FB60F9211241F932F9322
:1010C0003F934F935F936F937F938F939F93AF93D0
:1010D000BF93EF93FF939CB19D3041F080912F011E
:1010E000E82FF0E0E651FF4F9083C2C0E0912F015E
:1010F000F0E0E651FF4F908380912F01813009F598
:101100008091EA008E3341F410926000939A8091AE
:10111000E70088608093E7008091EA00853419F445
:1011200082E0809360008091EA00853619F483E0C4
:10113000809360008091EA00833509F0B8C08EE0AA
:10114000B4C080912F01823009F06EC08091EA0016
:101150008E3469F48091EB00843449F481E080930B
:101160006000939A8091E70088608093E700809107
:10117000EA00833469F48091EB00863449F484E01A
:1011800080936000939A8091E70088608093E700E5
:101190008091EA00823439F48091EB00833419F4B1
:1011A00085E0809360008091EA00843439F4809176
:1011B000EB00863419F486E0809360008091EA00A9
:1011C000863439F48091EB00893419F487E08093F8
:1011D00060008091EA00823539F48091EB008F3411
:1011E00019F488E0809360008091EA00863439F435
:1011F0008091EB008F3419F489E080936000809136
:10120000EA008E3439F48091EB00853419F48AE0D9
:10121000809360008091EA00863401F58091EB00B4
:101220008E34E1F48BE018C080912F01833021F5DA
:101230008091EA00843491F48091EC00823371F45F
:101240008091EB00843419F482E1809360008091F6
:10125000EB00823519F484E1809360008091EA000C
:10126000843529F58091EB00803209F580912F01BA
:101270008F5F80932F010EC180912F018430B9F4CC
:101280008091EA00843599F48091EB00803279F402
:101290003091EC002091ED00922F80E0830F911DA2
:1012A00090932C0180932B018FE0809360008091BC
:1012B000EA00803599F58091EB00803279F582E083
:1012C00080932F0120E00EC080912F01E82FF0E0E5
:1012D000E651FF4F9081AE59BF4F9C932F5F8F5FB8
:1012E00080932F01E0912F01F0E0E651FF4F108134
:1012F000A22FB0E01D3041F7AE59BF4F1C9280E0E5
:101300006CE04CE0D8D88091E7008F7E8093E700B6
:1013100081E080932E0110936000BAC080912E016D
:10132000882309F4B5C080912E01833009F45FC091
:10133000843038F4813009F4A3C0823009F0A8C0A9
:1013400007C0843009F49CC0853009F0A1C09EC05C
:1013500080912E018F5F80932E0110923201809137
:10136000EA008D3009F494C080912F018150809360
:101370002F0180E28093620080936300E2E00EC060
:1013800080912F01E82FF0E0E651FF4F9081AE5998
:10139000BF4F9C93E32F815080932F0180912F01A9
:1013A000AE2FB0E03E2F3F5F882351F7E0912F0131
:1013B000F0E0E651FF4F8081AE59BF4F8C93E32F91
:1013C000F0E0EE59FF4F20E22083832F8F5FE82F5C
:1013D000F0E0EE59FF4F9DE290838F5FE82FF0E041
:1013E000EE59FF4F20838F5F8093320151C080916F
:1013F0002E018F5F80932E018091EA008D30E9F1FC
:10140000809132018823C9F12091320180912F010E
:101410000BC080912F01E82FF0E0E651FF4F908143
:10142000AE59BF4F9C932F5F815080932F018091C5
:101430002F01A22FB0E0882361F7E0912F01F0E0A7
:10144000E651FF4F8081AE59BF4F8C9320933201FC
:10145000209331018091E7008F7D8093E7008BE03E
:1014600080932D018091E70080628093E700809156
:10147000E70080618093E7000BC01092320108C042
:1014800080912E018F5F80932E0102C010922E0159
:1014900010922F01FF91EF91BF91AF919F918F918A
:1014A0007F916F915F914F913F912F911F910F907D
:1014B0000FBE0F901F901895FF921F939598969AC4
:1014C0008D9A8B9A8E9A8C98949A84B3807C84BBE4
:1014D000AC9AAD9A85B38F6085BB8EB58A608EBDA0
:1014E00088EA91E69BBD8ABD89B7806189BF10BC3F
:1014F00089E189B988E98AB986E880BD849B04C0FE
:1015000088E080933E0102C010923E01109240019B
:101510008FEF80933A0184E083BF89B7816089BFF0
:1015200085B78C7F816085BF8BB780648BBF8CE073
:1015300067D780E062E471E064D888E06AE471E033
:1015400060D880E162E571E05CD888E16AE571E02D
:1015500058D880E262E671E054D888E26AE671E029
:1015600050D880E362E771E04CD888E36AE771E025
:1015700048D816D70D6083E08093E80010923601BA
:1015800010923701109261008091E7008E7F809366
:10159000E7008091E7008D7F8093E7008091E7006E
:1015A0008B7F8093E7008091E70088608093E7005D
:1015B0008091E7008F7E8093E7008091E7008F7D28
:1015C0008093E7008091E7008F7B8093E700809114
:1015D000E7008F778093E7008EE18093E900109217
:1015E000350110922C0110922B018FEF8093600037
:1015F00010922E0110922D011092320110923101A1
:10160000789485E490E0EFD687E590E0ECD688EA20
:1016100091E624E630E0F9013197F1F70197D9F727
:1016200088EA91E624E630E0F9013197F1F7019775
:10163000D9F7BDDBFF24F3941FEF1ADC00FF32C0A3
:10164000809136018430E1F0853038F4823081F0C9
:10165000833090F4813031F507C08630E9F0863070
:1016600098F08830F9F414C08093610017DB17C03C
:10167000F092610034DA13C0F092610060DA0FC0BA
:10168000F092610015DA0BC0F0926100FAD907C040
:10169000F0926100D6DA03C0F092610093DA08603C
:1016A0001092360180913601873031F4F09261005A
:1016B0007EDB086010923601809160008E3009F464
:1016C00064C08F3048F48430D9F18D3009F44CC0B7
:1016D000813009F074C008C0823141F1843151F089
:1016E0008F3009F06CC064C080E061E04FD68CEDB3
:1016F00090E005C080E061E049D68DEE90E073D6C1
:101700008091E7008E7F8093E7008091E7008D7FD6
:101710008093E7008091E7008B7F8093E7008091C2
:10172000E7008F7E8093E700086047C080E061E0BB
:101730002DD68FE091E057D68091E7008460EDCF01
:1017400080E061E023D680E291E04DD68091E70011
:101750008E7F8093E7008091E7008D7F8093E70084
:101760008091E7008F7E21C089E060E00FD681E0A4
:101770001DD68091E70081608093E7008091E700AB
:101780008D7F8093E7001BD818C089E060E0FED50C
:1017900080E00CD68BE990E026D68091E7008E7F22
:1017A0008093E7008091E7008D7F8093E70005C07C
:1017B00080912B0190912C01A9D81093600031D910
:1017C0001AD88091E70083FF02C0939A36CF93988E
:1017D00034CF991B79E004C0991F961708F0961B27
:1017E000881F7A95C9F780950895AA1BBB1B51E104
:1017F00007C0AA1FBB1FA617B70710F0A61BB70B81
:10180000881F991F5A95A9F780959095BC01CD0125
:061810000895F894FFCFDB
:00000001FF
